:040000008A017D28CC
:08000800F700F70E030EF800EB
:10001000040EF9000A0EFA008A010B1C6028030185
:1000200083120313061A0130FB007B087D020130A6
:1000300003190301FF39031926287C08003C01300D
:10004000031D0301FF39031926280130003C031961
:1000500037287B08FD000130FC00831203131010C9
:100060000E0883120313AC000F08AD001014030137
:1000700083120313061B0130FB007B0820020130B2
:1000800003190301FF3903194E287F08003C013092
:10009000031D0301FF3903194E280130003C0319E9
:1000A0005F287B0883120313A0000130FF00831236
:1000B000031310100E08AE000F08AF0010140B1041
:1000C000831203130C0883120313A200221C752849
:1000D00005307E02031CFE0A053083120313210241
:1000E000031CA10A831203130C107A0E8A00790EE6
:1000F0008400780E8300770E0900831203139701A2
:100100009D0183160313FB3092008312031300300A
:1001100095009B00971217129D121D128316031350
:1001200007118710831203139201910183120313A5
:10013000121583120313971517159D151D1583129C
:10014000031390011014831203130C10831603136E
:100150000C148312031383120313850183160313F4
:1001600006309F00831603138316051085100511B2
:1001700085118512831203138312860183160313DC
:100180008316061606170B108B150B178B17831289
:10019000A801FE01A101A301A401FC01FF017C084B
:1001A0000319C729831203132308013C0130031DDF
:1001B0000301FF390319E5287D08003C0130031DC8
:1001C0000301FF390319E5280130003C0319A62972
:1001D00083120313A3012D08F0002C08B800700847
:1001E000B900390837020130031CFE280030031D16
:1001F000FE28380836020130031803018312031366
:10020000A70027080319112936083802F10037081A
:10021000031C013E3902F0007108B0007008B10003
:100220002A298312031336083802F1003708031C09
:10023000013E3902F0007108B2007008B3003308C3
:10024000F000FF30F0073208FF3E0318F00AB0005C
:100250007008B1009030831203133002F1000130B6
:10026000031C013E3102F0007108B2007008B300B7
:100270003308F0003208B0007008B10031080B3CC0
:100280000130031C4B290030031D4B293008B83CBA
:1002900001300318030183120313A5002930310232
:1002A0000130031C5B290030031D5B290430300240
:1002B00001300318030183120313A6002508FF3938
:1002C000031967292608FF39031967290130003C03
:1002D0000319C629FE0112308312031331020130C3
:1002E000031C7A290030031D7A295C30300201306A
:1002F00003180301003C031983295C3083120313A4
:10030000B0001230B100831203133108213C0130D8
:10031000031C92290030031D92293008FC3C013057
:1003200003180301003C03199B29FC3083120313BB
:10033000B0002130B100831203133108F0003008FF
:10034000BE007008BF000130A800C6298312031345
:100350002308003C0130031D0301FF390319B929AB
:100360007D08013C0130031D0301FF390319B92940
:100370000130003C0319C629013083120313A30086
:100380002D08F0002C08B6007008B700FC017F08AB
:100390000319AD2A831203132408013C0130031D05
:1003A0000301FF390319DD292008003C0130031D3A
:1003B0000301FF390319DD290130003C03198C2AA0
:1003C00083120313A4012F08F0002E08BC0070084C
:1003D000BD003D083B020130031CF6290030031D1F
:1003E000F6293C083A020130031803018312031373
:1003F000A70027080319092A3A083C02F1003B0824
:10040000031C013E3D02F0007108B0007008B1000D
:10041000222A831203133A083C02F1003B08031C12
:10042000013E3D02F0007108B2007008B3003308CD
:10043000F000FF30F0073208FF3E0318F00AB0006A
:100440007008B1008312031331080B3C0130031C08
:10045000312A0030031D312A3008B83C013003181E
:10046000030183120313A500293031020130031C5C
:10047000412A0030031D412A0430300201300318A4
:10048000030183120313A6002508FF3903194D2A1F
:100490002608FF3903194D2A0130003C0319AC2A04
:1004A00083120313A101123031020130031C602AB0
:1004B0000030031D602A5C30300201300318030154
:1004C000003C0319692A5C3083120313B000123018
:1004D000B100831203133108213C0130031C782A38
:1004E0000030031D782A3008FC3C0130031803015A
:1004F000003C0319812AFC3083120313B000213021
:10050000B100831203133108F0003008C0007008F6
:10051000C1000130A800AC2A831203132408003C58
:100520000130031D0301FF3903199F2A2008013CF4
:100530000130031D0301FF3903199F2A0130003CDC
:100540000319AC2A013083120313A4002F08F00012
:100550002E08BA007008BB00FF0183120313A90123
:100560003F08193C0130031CBD2A0030031DBD2A81
:100570003E08F53C013003180301FF390319D32A63
:100580001A30831203133F020130031CCF2A0030BC
:10059000031DCF2A63303E02013003180301FF39E7
:1005A0000319D32A0130FF390319E92A83120313EF
:1005B0004108193C0130031CE52A0030031DE52ADF
:1005C0004008F53C013003180301FF390319E92AFB
:1005D0000130FF390319FF2A1A3083120313410235
:1005E0000130031CFB2A0030031DFB2A633040024C
:1005F000013003180301FF390319FF2A0130003CC1
:100600000319062B013083120313A90005307E0263
:100610000130031C0301FF39031D182B0530831221
:10062000031321020130031C0301FF390319192BA5
:100630000130FF39031D262B831203132908013CC7
:100640000130031D0301FF390319272B0130003C42
:100650000319362B8312031305108510051185111C
:1006600085128312031395019B01C72D8312031377
:10067000051428080319C72DA8015C303E02F100BB
:100680001230031C013E3F02F0007108B2007008F6
:10069000B3005C304002F1001230031C013E410205
:1006A000F0007108B0007008B1003308F0003108A4
:1006B000F007320830070318F00AB4007008B500DC
:1006C000073035020130031C6D2B0030031D6D2BEC
:1006D000D0303402013003180301003C0319782B99
:1006E0000730F000D03083120313B4007008B50057
:1006F000831203133508173C0130031C872B00308D
:10070000031D872B3408703C013003180301003CA3
:100710000319922B1730F000703083120313B400CA
:100720007008B500D030831203133402F100073093
:10073000031C013E3502F0007108B2007008B300DE
:100740003308073C0130031CAD2B0030031DAD2BDB
:100750003208DC3C013003180301003C0319C12BB3
:100760008312031385128515DC303202F100073045
:10077000031C013E3302F0007108B0007008B100A4
:10078000EA2B07308312031333020130031CD02BF2
:100790000030031DD02BC430320201300318030196
:1007A000003C0319E42B83120313851185163208CC
:1007B000C43CF1003308031C013E073CF000710803
:1007C000B0007008B100EA2B831203138511851263
:1007D000B001B101831203133108F0003008B200F8
:1007E0007008B3003208F1003308F000F00CF10C8F
:1007F000700CF10C3F39F0007108F101B000700885
:10080000B100F001F1013008F2003108F30041308D
:10081000F400F5011030F600F30CF20C031C162C5A
:100820007508F0077408F1070318F00A0310F40DB7
:10083000F50DF60B0C2C710883120313B20070082F
:10084000B3003208F1003308F000F00CF10CF00CAA
:10085000F10CF00CF10CF00CF10CF00CF10CF00CB4
:10086000F10C700CF10C0139F0007108F101B000CD
:100870007008B1003008AA002A08FB3C0318422C7B
:10088000FB30AA00831203132A08FC3CAB0083123E
:1008900003132B089B005C303E02F1001230031C56
:1008A000013E3F02F0007108B0007008B10031084D
:1008B000F0000F30F0073008A03E0318F00AB20035
:1008C0007008B3005C304002F1001230031C013E9E
:1008D0004102F0007108B0007008B1003308F00068
:1008E0003108F007320830070318F00AB400700826
:1008F000B500A0303402F1000F30031C013E350278
:10090000F0007108B0007008B1000730310201300A
:10091000031C922C0030031D922CD0303002013089
:1009200003180301003C03199D2C0730F000D03060
:1009300083120313B0007008B1008312031331084F
:10094000173C0130031CAC2C0030031DAC2C3008CC
:10095000703C013003180301003C0319B72C173019
:10096000F000703083120313B0007008B100D03073
:10097000831203133002F1000730031C013E3102E1
:10098000F0007108B2007008B3003F08F0000F30AB
:10099000F0073E08A03E0318F00AB2007008B3004A
:1009A00040083202F1004108031C013E3302F0000E
:1009B0007108B0007008B100073031020130031C2B
:1009C000E92C0030031DE92CD0303002013003182F
:1009D0000301003C0319F42C0730F000D0308312DF
:1009E0000313B0007008B100831203133108173CE1
:1009F0000130031C032D0030031D032D3008703C13
:100A0000013003180301003C03190E2D1730F000CC
:100A1000703083120313B0007008B100D03083121D
:100A200003133002F1000730031C013E3102F000D5
:100A30007108B2007008B3003308073C0130031C92
:100A4000292D0030031D292D3208DC3C013003180C
:100A50000301003C03193D2D831203130511851476
:100A6000DC303202F1000730031C013E3302F0009B
:100A70007108B0007008B100662D073083120313AF
:100A800033020130031C4C2D0030031D4C2DC430AB
:100A90003202013003180301003C0319602D831258
:100AA0000313851005153208C43CF1003308031CFC
:100AB000013E073CF0007108B0007008B100662DDF
:100AC0008312031385100511B001B10183120313C2
:100AD0003108F0003008B2007008B3003208F100AD
:100AE0003308F000F00CF10C700CF10C3F39F00001
:100AF0007108F101B0007008B100F001F101300897
:100B0000F2003108F3004130F400F5011030F60036
:100B1000F30CF20C031C922D7508F0077408F10712
:100B20000318F00A0310F40DF50DF60B882D71086B
:100B300083120313B2007008B3003208F1003308C7
:100B4000F000F00CF10CF00CF10CF00CF10CF00CCE
:100B5000F10CF00CF10CF00CF10C700CF10C0139F3
:100B6000F0007108F101B0007008B1003008AA006F
:100B70002A08FB3C0318BE2DFB30AA008312031386
:100B80002A08FC3CAB00831203132B089500640079
:020B9000CF286C
:00000001FF
